:20000000011002303110203030103038003030003030003030003030003030003020001024
:200020003000303000300000303030205030300030103000000000001020003021000000AF
:20004000201000102010302020200000202000300020200030001030000010100010300020
:200060000010303000002030100020000010001030203020001130102010102002000020FD
:2000800000000020000010200001302000302001300000200010000000200030302000006E
:2000A000101000300000103000305030300020302000202010310000011010391000200055
:2000C000300000303030301010003010103020000020201000202010101000201018103028
:2000E00020003010303000303030001030001000002120000020202010301010000022003D
:200100001010102000101020000000111000100000101030000000002020302030001020DE
:2001200000101010100010100000002020000000001020201020000010000000200800085F
:2001400010002020200020001000000020002000002020003020000020101000202020008F
:20016000002010003020002030001010102000202110010100000000202002001021201069
:2001800000002000000000201020101010001018000000000000000010000000102010083F
:2001A00020200010002020300000200000002010110820100020100010010000002109205B
:2001C0001000002000000000000000002010301000000000000030000000000001201020FE
:2001E00000000000000010201020100010000000200000001100100000000001200000001D
:2002000000200000000000001010100012102200000000000000000010000000000000003A
:200220000000202000002000110000002000001001020000110100080000010010000200ED
:2002400000000020000000000000100002001010000000000010000010000000100002001A
:2002600002003000100030203020000000000020000000000008010010000000000008203B
:2002800000000000000010201000100000101008002010000000100010001010100800005E
:2002A0001000003030001000000000283000101000000001000800080001000008080028FC
:2002C0000020300000201100100010011108100800000000100030000000000010083808B3
:2002E000203000300000000010102020002800100000111B0018010010081020110919091D
:2003000030200000001030003020000000083000010000010000000000003000300810004B
:200320000000000010001000002010000000101800100110000000001010100000000000F4
:200340000000100010003000200008202008200800001000100010002010000031103000E4
:20036000000000301030200000003010001000383000200010100000002010002012001083
:2003800010000020000010101000103000081000100000000000001000300030000800001D
:2003A00010102020002000100000101020100020303830001008183030302008080030186D
:2003C0003020000000303000100010182020301010200010001030001010000020212000B4
:2003E000101000300010101000202000000010100020300000000010101000040024000075
:20040000001000100020003000000000100820180020001000001010001000000010200884
:20042000001000102000001000101000100020003010101010200030103030103020003854
:200440000010300010100000200020002010003000101010000020000020101000103000CC
:2004600000000010100000000020000000100010001000100008300010000038001000006C
:200480003000100000303010303030203030302830000000201010102030302010101010E4
:2004A0000020202010200000200030202000202020000030101000101008101000003020D4
:2004C0000030200030302010300010103020101010102000000020001000002000103000AC
:2004E0003010301010203000103010000020000000100010000000000000302000081030F4
:200500002000001000001000000030200000102820300020000010200000200000203028DB
:200520000000000020000020200010000020200800000000000000001000100020001008AB
:200540001000000000002010002000100000200800002000000000002000100000000000B3
:20056000000000000000001020301010000020000820002028000000020210200000112006
:2005800000001030002020003000202000000000000000000000000000000000200000004B
:2005A000300000000020000000000000000000200801012000020000121013000019280128
:2005C0002020002200100000000010002208001920002100002000000001010200000001F0
:2005E00010000000000000001000000000000008020000200000012001092900000200005B
:2006000000000010002010000020101010221010002000000000200010000002012030283D
:200620001000201000000000000000000020000003080001212019021801010220020000B4
:200640002008000000001000000010000800100800000020000001000800290001080020B7
:20066000000000002030000000001100100000000300080801000100120301021208080AB0
:200680000800000020020000001000000800102000000000000000080000200001000119A5
:2006A0000000100000000000103000001008101001000003000120080120022900213902DD
:2006C0000000002020002018200800080010200000010000200020000000200800083000A1
:2006E0002020000020000000201020280000202000080001200220080100020A010300225C
:20070000203000202000100010000039300010002020000000080000000012000008000A44
:20072000000000100020002008002010101800002100000801002008202008200100110835
:20074000000020082020302000201000282200100801002200000020000811201028002873
:200760002000000030200000003030200020002830202028210021000808082010020820F5
:200780002000000010001000200020201000002800002000000030020000002032000000DD
:2007A00010001000302000000020000000200008000000000020020002200020010000001C
:2007C0000020001000200020010000201810100000000000202000002000000000200000D0
:2007E000000000002000001000200000302000000000000000000000000000000000000059
:00000001FF
